:020000040800F2
:1000000000000220E52F00086D2F00086F2F000868
:10001000712F0008732F0008752F000800000000E2
:10002000000000000000000000000000E1230008C4
:10003000772F00080000000081240008792F0008B5
:1000400035300008353000083530000835300008FC
:1000500035300008353000083530000835300008EC
:1000600035300008353000083530000835300008DC
:1000700035300008353000083530000835300008CC
:1000800035300008353000083530000835300008BC
:1000900035300008353000083530000835300008AC
:1000A000353000083530000835300008353000089C
:1000B000353000083530000835300008353000088C
:1000C000353000083530000835300008353000087C
:1000D0003530000835300008852F0008353000081D
:1000E000353000083530000835300008353000085C
:1000F000353000083530000835300008353000084C
:10010000353000083530000835300008353000083B
:10011000353000083530000835300008353000082B
:10012000353000083530000835300008353000081B
:1001300035300008000000000000000035300008E5
:1001400035300008353000083530000835300008FB
:1001500035300008353000083530000835300008EB
:1001600035300008353000083530000835300008DB
:100170003530000835300008353000080000000038
:100180000000000035300008000000000000000002
:100190003530000800000000000000003530000885
:1001A00000000000000000000000000035300008E2
:1001B000353000083530000835300008353000088B
:0401C00035300008CE
:1001D00010B5054C237833B9044B13B10448AFF381
:1001E00000800123237010BD940200200000000055
:1001F000303200080C4B43B10C480D4910B5AFF339
:1002000000800C48036823B910BD0A48036833B95D
:100210007047094B002BF7D0BDE810401847064B3C
:10022000002BF5D0184700BF000000003032000856
:1002300098020020940200200000000053B94AB93F
:10024000002908BF00281CBF4FF0FF314FF0FF30DE
:1002500000F07AB9ADF1080C6DE904CE00F006F8B3
:10026000DDF804E0DDE9022304B070472DE9F04732
:100270008C460D460446089E002B51D18A421746F3
:100280006DD9B2FA82FEBEF1000F0BD0CEF1200C78
:1002900001FA0EF520FA0CFC02FA0EF74CEA050CF6
:1002A00000FA0EF44FEA174A250CBCFBFAF81FFAC5
:1002B00087F90AFB18CC45EA0C4508FB09F3AB4269
:1002C0000AD9ED1908F1FF3280F02381AB4240F2E8
:1002D0002081A8F102083D44ED1AA4B2B5FBFAF062
:1002E0000AFB105544EA054400FB09F9A14509D968
:1002F000E41900F1FF3380F00A81A14540F2078143
:1003000002383C44A4EB090440EA08400021002ED6
:1003100061D024FA0EF4002334607360BDE8F087E6
:100320008B4207D9002E54D0002186E821000846D0
:10033000BDE8F087B3FA83F1002940F08E80AB422C
:1003400002D3824200F2FA80841A65EB0305012091
:10035000AC46002E3FD086E81010BDE8F08712B9F9
:100360000127B7FBF2F7B7FA87FEBEF1000F34D1D1
:10037000EB1B3A0C1FFA87FC0121B3FBF2F8250CAA
:1003800002FB183345EA03450CFB08F3AB4207D9DF
:10039000ED1908F1FF3002D2AB4200F2D180804665
:1003A000ED1AA3B2B5FBF2F002FB105543EA054487
:1003B0000CFB00FCA44507D9E41900F1FF3302D27D
:1003C000A44500F2B8801846A4EB0C0440EA0840AB
:1003D0009DE731463046BDE8F087CEF1200405FAAE
:1003E0000EF307FA0EF720FA04F83A0C25FA04F493
:1003F00048EA0308B4FBF2F14FEA184502FB114446
:100400001FFA87FC45EA044501FB0CF3AB4200FAF6
:100410000EF409D9ED1901F1FF3080F08A80AB426A
:1004200040F2878002393D44EB1A1FFA88F5B3FB8E
:10043000F2F002FB103345EA034500FB0CF3AB423C
:1004400007D9ED1900F1FF386FD2AB426DD90238F0
:100450003D44EB1A40EA01418FE7C1F1200722FA3F
:1004600007F88B4005FA01F448EA030320FA07FE77
:100470004FEA134CFD404EEA040EB5FBFCF94FEA7F
:100480001E440CFB19551FFA83F844EA054509FB85
:1004900008F4AC4202FA01F200FA01FA08D9ED18A8
:1004A00009F1FF3043D2AC4241D9A9F102091D4400
:1004B0002D1B1FFA8EFEB5FBFCF00CFB10554EEA0F
:1004C000054400FB08F8A04507D9E41800F1FF3502
:1004D00029D2A04527D902381C4440EA0940A4EBA0
:1004E0000804A0FB02894C45C6464D4615D312D0E0
:1004F00056B1BAEB0E0364EB050404FA07F7CB40E0
:100500001F43CC40376074600021BDE8F087184677
:10051000F8E69046E0E6C245EAD2B8EB020E69EB97
:1005200003050138E4E72846D7E7404691E78146CE
:10053000BEE7014678E702383C4445E7084608E74D
:10054000A8F102083D442BE7704700BF10B50446F0
:100550000E4B18784FF47A73B3FBF0F30C4A106823
:10056000B0FBF3F000F092F868B90F2C01D901202C
:1005700010BD002221464FF0FF3000F049F8034B38
:100580005C60002010BD012010BD00BF00000020F5
:10059000C000002008B50B4B1A6842F400721A60C4
:1005A0001A6842F480621A601A6842F480721A6013
:1005B000032000F01BF80F20FFF7C8FF02F02CFC0F
:1005C000002008BD003C0240034A1168034B1B7821
:1005D0000B441360704700BF34400020000000202F
:1005E000014B1868704700BF34400020074AD368A9
:1005F00023F4E0631B041B0C000200F4E0601843CA
:1006000040F0BF6040F40030D060704700ED00E083
:1006100030B4164BDB68C3F30223C3F10704042C88
:1006200028BF04241D1D062D17D9033B012505FAFB
:1006300004F4013C2140994005FA03F3013B1340C7
:10064000194300280BDB0901C9B200F1604000F535
:10065000614080F8001330BC70470023E6E700F0EB
:100660000F000901C9B2024B1954F4E700ED00E094
:1006700014ED00E0420900F01F00012303FA00F02E
:10068000014B43F82200704700E100E00138B0F16F
:10069000807F0AD2064B5860F021064A82F8231068
:1006A0000020986007221A6070470120704700BF41
:1006B00010E000E000ED00E0042805D0054A1368D2
:1006C00023F0040313607047024A136843F00403E5
:1006D0001360704710E000E090F83530DBB2022B79
:1006E00003D08023436501207047052380F835300F
:1006F0000268136823F001031360002070470000B4
:10070000F0B583B0002498E04FEAD40E0EF1080E45
:1007100050F82E2004F00706B6000F27B74022EA53
:1007200007020F6907FA06F6324340F82E2094E0DC
:1007300086681640CF6807FA0EF73E438660466823
:1007400026EA03034E68C6F30016A640334343600F
:10075000C3681A408B6803FA0EF31A43C2604B68F1
:1007600013F0805F68D000230193514B5A6C42F420
:1007700080425A645B6C03F480430193019BA3089D
:100780009E1C4C4A52F8262004F003064FEA860EBF
:100790000F2606FA0EF622EA0602474FB84279D033
:1007A000464EB04278D006F58066B04276D006F567
:1007B0008066B04274D006F58066B04272D006F50D
:1007C0008066B04270D006F58066B04260D00726E1
:1007D00006FA0EF632430233364E46F82320384BE3
:1007E0001A68EB4302EA03064F6817F4803F01D012
:1007F00045EA0206324A1660526803EA02064F686A
:1008000017F4003F01D045EA02062D4A566092686F
:1008100003EA02064F6817F4801F01D045EA02067A
:10082000274A9660D26813404E6816F4001F01D024
:1008300045EA0203224AD36001340F2C36D8012343
:10084000A3400A6803EA0205AB42F5D14A68022ACE
:100850003FF45AAF122A3FF457AF06684FEA440EEE
:10086000032202FA0EF2D24316404F6807F0030744
:1008700007FA0EF73E4306604E68771E012F7FF69B
:1008800057AF112E3FF454AF122E7FF461AF4FE7F4
:1008900006269DE700269BE7012699E7022697E7B3
:1008A000032695E7042693E7052691E703B0F0BDFC
:1008B00000380240003801400000024000040240BD
:1008C000003C0140002800F09D8070B504464F4B6D
:1008D0001B6803F00F038B4209D2CBB24B4A137053
:1008E000136803F00F03994201D0012070BD236803
:1008F00013F0020F17D013F0040F04D0444A93688A
:1009000043F4E0539360236813F0080F04D0404A87
:10091000936843F4604393603D4A936823F0F00387
:10092000A068034393600D46236813F0010F32D093
:100930006368012B21D09A1E012A25D9344A1268F6
:1009400012F0020F60D032498A6822F0030213438A
:100950008B60FFF745FE06462D4B9B6803F00C03AA
:100960006268B3EB820F16D0FFF73AFE801B41F2AC
:1009700088339842F0D9032070BD254A126812F4DA
:10098000003FE0D1012070BD214A126812F0007FC3
:10099000D9D1012070BD1D4B1B6803F00F039D4290
:1009A00009D2EAB2194B1A701B6803F00F039D427B
:1009B00001D0012070BD236813F0040F06D0144A43
:1009C000936823F4E053E1680B439360236813F0CA
:1009D000080F07D00E4A936823F46043216943EA65
:1009E000C103936000F040F8094B9B68C3F3031305
:1009F000084AD35CD840084B18600F20FFF7A6FDCB
:100A0000002070BD01207047012070BD003C0240F5
:100A10000038024048320008C0000020014B18682E
:100A2000704700BFC000002008B5FFF7F7FF044B78
:100A30009B68C3F38223034AD35CD84008BD00BF40
:100A4000003802405832000808B5FFF7E7FF044BB2
:100A50009B68C3F34233034AD35CD84008BD00BF50
:100A60000038024058320008F8B5444B9B6803F048
:100A70000C03082B05D00C2B41D0042B7BD0404815
:100A8000F8BD3E4B5A6802F03F025B6813F4800FDA
:100A900012D03A4B5968C1F3881100233948A1FBA1
:100AA0000001FFF7CBFB354B5B68C3F30143013318
:100AB0005B00B0FBF3F0F8BD304B5B68C3F3881309
:100AC0001E4600275C010025E41A65EB0705A90115
:100AD00041EA9461A001001B61EB0501CB0043EAF0
:100AE0005073C400A01943EB07018B0243EA9053F3
:100AF0008402204619460023FFF7A0FBD3E71F4BD3
:100B00005A6802F03F025B6813F4800F10D01B4B51
:100B10005968C1F3881100231A48A1FB0001FFF7AF
:100B20008DFB164B5B68C3F30273B0FBF3F0F8BDAB
:100B3000124B5B68C3F388131E4600275C01002537
:100B4000E41A65EB0705A90141EA9461A001001BC5
:100B500061EB0501CB0043EA5073C400A01943EBDD
:100B600007018B0243EA9053840220461946002372
:100B7000FFF764FBD5E70348F8BD00BF003802402B
:100B80000024F40040787D0170B582B0044603680B
:100B900013F0010F41D0A64B9B6803F00C03042B0C
:100BA00032D0A34B9B6803F00C03082B27D0A04B3B
:100BB0009B6803F00C030C2B59D06368B3F5803F9E
:100BC0005BD0B3F5A02F5ED0994B1A6822F4803227
:100BD0001A601A6822F480221A606368002B5CD0C5
:100BE000FFF7FEFC0546924B1B6813F4003F14D13F
:100BF000FFF7F6FC401B6428F5D903209DE18C4BE0
:100C00005B6813F4800FD2D0894B1B6813F4003F4C
:100C100003D06368002B00F08D81236813F0020F6E
:100C200067D0834B9B6813F00C0F4AD0804B9B68B6
:100C300003F00C03082B3FD07D4B9B6803F00C03A3
:100C40000C2B48D0E368002B74D00122794B1A603A
:100C5000FFF7C6FC0546764B1B6813F0020F60D108
:100C6000FFF7BEFC401B0228F5D9032065E1704B5D
:100C70005B6813F4800FA0D0C6E76D4A136843F495
:100C800080331360A9E76A4B1A6842F480221A6025
:100C90001A6842F480321A609FE7FFF7A1FC05460C
:100CA000634B1B6813F4003FB7D0FFF799FC401B60
:100CB0006428F5D9032040E15D4B5B6813F4800F95
:100CC000BAD15B4B1B6813F0020F0AD0E368012B0B
:100CD00007D0012031E1564B5B6813F4800FB1D18E
:100CE000EFE7534A136823F0F803216943EAC1038D
:100CF0001360236813F0080F40D0636963B30122C7
:100D00004D4B1A60FFF76CFC0546494B5B6F13F0C7
:100D1000020F33D1FFF764FC401B0228F5D90320F2
:100D20000BE1434A136823F0F803216943EAC10346
:100D30001360DEE700223F4B1A60FFF751FC0546C7
:100D40003B4B1B6813F0020FD3D0FFF749FC401B4D
:100D50000228F5D90320F0E00022374B1A60FFF794
:100D60003FFC0546324B5B6F13F0020F06D0FFF7D6
:100D700037FC401B0228F5D90320DEE0236813F07E
:100D8000040F79D02A4B1B6C13F0805F33D1002302
:100D90000193274B1A6C42F080521A641B6C03F0CB
:100DA00080530193019B0125244B1B6813F4807F22
:100DB00023D0A368012B34D0052B41D01C4B1A6FD4
:100DC00022F001021A671A6F22F004021A67A36860
:100DD000002B3FD0FFF704FC0646154B1B6F13F0AA
:100DE000020F48D1FFF7FCFB801B41F28833984289
:100DF000F3D90320A1E00025D6E7104A136843F495
:100E000080731360FFF7ECFB06460C4B1B6813F472
:100E1000807FCED1FFF7E4FB801B0228F5D90320A9
:100E20008BE0034A136F43F001031367CFE700BF62
:100E30000038024000004742800E474200700040E8
:100E4000404B1A6F42F004021A671A6F42F0010217
:100E50001A67BCE7FFF7C4FB06463A4B1B6F13F05B
:100E6000020F08D0FFF7BCFB801B41F28833984289
:100E7000F3D9032061E0E5B9A369002B5CD0314AC6
:100E8000926802F00C02082A59D0022B17D00022D7
:100E90002D4B1A60FFF7A4FB04462A4B1B6813F086
:100EA000007F45D0FFF79CFB001B0228F5D90320EB
:100EB00043E0244A136C23F080531364DCE70022E0
:100EC000214B1A60FFF78CFB05461E4B1B6813F085
:100ED000007F06D0FFF784FB401B0228F5D90320D2
:100EE0002BE0E369226A1343626A43EA8213A26A2F
:100EF0005208013A43EA0243E26A43EA0263226B80
:100F000043EA02730F4A536001220F4B1A60FFF746
:100F100067FB04460B4B1B6813F0007F06D1FFF7FD
:100F20005FFB001B0228F5D9032006E0002004E047
:100F3000002002E0012000E0002002B070BD01208E
:100F4000FBE700BF003802406000474230B4036A4C
:100F500023F001030362036A4468826922F073028A
:100F60000D682A4323F002038D682B430F4DA842DE
:100F70001AD005F58065A84214D000255DB123F094
:100F80000803CD682B4323F0040324F440744D6917
:100F90002C438D692C43446082614A68426303623A
:100FA00030BC70470125E9E70125E7E70000014073
:100FB00030B4036A23F480730362036A4468C2692D
:100FC00022F073020D682A4323F400738D6843EA0C
:100FD0000523114DA8421DD005F58065A84217D004
:100FE000002575B123F40063CD6843EA052323F49B
:100FF000806324F440544D6944EA05148D6944EA41
:1010000005144460C2614A68C263036230BC704721
:101010000125E6E70125E4E70000014030B4036A5A
:1010200023F480530362036A4468C26922F4E642EF
:101030000D6842EA052223F400538D6843EA053324
:101040000C4DA84213D005F58065A8420DD00025AF
:1010500025B124F480444D6944EA85144460C2619A
:101060004A680264036230BC70470125F0E701253D
:10107000EEE700BF000001400368454A90424AD0B5
:10108000B0F1804F49D0A2F57C42904247D002F5A2
:101090008062904245D002F58062904243D002F5D2
:1010A0007842904235D000221AB123F070034A688A
:1010B0001343374A90423AD0B0F1804F50D0A2F556
:1010C0007C4290424ED002F5806290424CD002F5B4
:1010D000806290424AD002F57842904248D002F5B0
:1010E0007052904246D002F58062904244D002F5A0
:1010F0008062904242D0A2F59832904240D002F5F0
:10110000806290423ED002F5806290420DD0002273
:101110000EE00122C8E70122C6E70122C4E701224E
:10112000C2E70122C0E70122BEE7012200E001225E
:101130001AB123F44073CA68134303608B68C36217
:101140000B688362124B984220D003F5806398426B
:101150001AD000230BB10B6903630123436170476D
:101160000122E5E70122E3E70122E1E70122DFE7CF
:101170000122DDE70122DBE70122D9E70122D7E7DF
:101180000122D5E70122D3E70123E3E70123E1E7C9
:1011900000000140A8B110B5044690F839305BB1A9
:1011A000022384F83930211D2068FFF765FF0123F1
:1011B00084F83930002010BD80F8383001F076FE18
:1011C000EEE701207047000030B4036A23F01003FB
:1011D0000362036A4468826922F4E6420D6842EAC7
:1011E000052223F020038D6843EA0513114DA84220
:1011F0001DD005F58065A84217D0002575B123F0F4
:101200008003CD6843EA051323F0400324F44064CF
:101210004D6944EA85048D6944EA8504446082612D
:101220004A688263036230BC70470125E6E7012506
:10123000E4E700BF0000014038B590F83830012BDA
:1012400066D00D460446012380F83830022380F82A
:1012500039300C2A1AD8DFE802F0071919192019B9
:1012600019193419191947000068FFF76FFE226831
:10127000936943F0080393612268936923F00403A0
:1012800093612268936929690B439361012384F870
:101290003930002084F8380038BD0068FFF794FF2B
:1012A0002268936943F4006393612268936923F48D
:1012B0008063936122689369296943EA01239361FA
:1012C000E4E70068FFF774FE2268D36943F008037F
:1012D000D3612268D36923F00403D3612268D36900
:1012E00029690B43D361D1E70068FFF797FE2268B5
:1012F000D36943F40063D3612268D36923F4806324
:10130000D3612268D369296943EA0123D361BDE728
:10131000022038BD10B4012303FA01F4036A23EA62
:1013200004030362036A8A40134303625DF8044BBB
:101330007047000010B5044601220068FFF7EAFF7D
:1013400023680C4A934212D002F5806293420CD07B
:1013500000221AB15A6C42F400425A64226813689F
:1013600043F001031360002010BD0122F1E70122C8
:10137000EFE700BF0000014010B5044600220068FE
:10138000FFF7C8FF2368174A934229D002F580620D
:10139000934223D000226AB1196A41F2111211421C
:1013A00008D1196A40F24442114203D15A6C22F426
:1013B00000425A642368196A41F21112114208D19D
:1013C000196A40F24442114203D11A6822F0010224
:1013D0001A60012384F83930002010BD0122DAE7B9
:1013E0000122D8E70000014090F83830012B22D0CC
:1013F00030B4012280F83820022380F839300468A4
:10140000636823F070036360046863680D682B43AE
:1014100063600468A36823F08003A3600468A36882
:1014200049680B43A36080F83920002380F83830E6
:10143000184630BC7047022070470268D36823F416
:101440009073D3600268536923F001035361202332
:1014500080F83A30704790F83930DBB2212B01D058
:10146000022070478368B3F5805F17D00268036A73
:10147000591C01621B785360C38C9BB2013B9BB229
:10148000C384DBB90268D36823F08003D3600268A9
:10149000D36843F04003D36000207047036A0268BA
:1014A0001B88C3F30803536003691BB9036A023343
:1014B0000362E1E7036A01330362DDE7002070475E
:1014C0002DE9F04704460268136923F44053C168CC
:1014D0000B4313610168CB6823F4164323F00C031C
:1014E00082680069024360690243E0690243134372
:1014F000CB602268536923F44073A1690B435361A5
:10150000E369B3F5004F62D0D4F80080BB4B984537
:1015100000F01B8103F58063984500F01681FFF70A
:1015200083FA00EB800000EB80006568AD00B0FB43
:10153000F5F5B34FA7FB05356D092E01FFF774FADA
:1015400000EB800000EB80006568AD00B0FBF5FAB1
:10155000FFF76AFA00EB800000EB80006568AD00E1
:10156000B0FBF5F5A7FB05356D094FF0640909FBE4
:1015700015A52D013235A7FB05356D0905F0F005E0
:101580003544FFF751FA00EB800000EB80006668FD
:10159000B600B0FBF6F6FFF747FA00EB800000EB71
:1015A000800063689B00B0FBF3F0A7FB00304009AC
:1015B00009FB10694FEA091909F13209A7FB09373C
:1015C000C7F343172F44C8F80870BDE8F087D4F874
:1015D000008003F1804303F5104398455CD003F588
:1015E0008063984558D0FFF71FFA00EB800000EBAE
:1015F000800065686D00B0FBF5F5814FA7FB0535F0
:101600006D092E01FFF710FA00EB800000EB80005F
:1016100065686D00B0FBF5FAFFF706FA00EB800095
:1016200000EB800065686D00B0FBF5F5A7FB0535A4
:101630006D094FF0640909FB15A5ED003235A7FBD4
:1016400005356D096D0005F4F8753544FFF7ECF9C3
:1016500000EB800000EB800066687600B0FBF6F6D9
:10166000FFF7E2F900EB800000EB800063685B00AD
:10167000B0FBF3F3A7FB03235B0909FB13694FEAF4
:10168000C90909F13209A7FB0937C7F342172F44EB
:10169000C8F80870BDE8F087FFF7D6F900EB8000C6
:1016A00000EB800065686D00B0FBF5F5544FA7FBBB
:1016B00005356D092E01FFF7C7F900EB800000EB3F
:1016C000800065686D00B0FBF5FAFFF7BDF900EB2F
:1016D000800000EB800065686D00B0FBF5F5A7FBAE
:1016E00005356D094FF0640909FB15A5ED0032358C
:1016F000A7FB05356D096D0005F4F8753544FFF756
:10170000A3F900EB800000EB800066687600B0FB78
:10171000F6F6FFF799F900EB800000EB80006368B4
:101720005B00B0FBF3F3A7FB03235B0909FB136921
:101730004FEAC90909F13209A7FB0937C7F3421774
:101740002F44C8F80870BDE8F087FFF77DF900EB7B
:10175000800000EB80006568AD00B0FBF5F5284F18
:10176000A7FB05356D092E01FFF76EF900EB800030
:1017700000EB80006568AD00B0FBF5FAFFF764F997
:1017800000EB800000EB80006568AD00B0FBF5F574
:10179000A7FB05356D094FF0640909FB15A52D015F
:1017A0003235A7FB05356D0905F0F0053544FFF727
:1017B0004BF900EB800000EB80006668B600B0FBE0
:1017C000F6F6FFF741F900EB800000EB800063685C
:1017D0009B00B0FBF3F3A7FB03235B0909FB136931
:1017E0004FEA091909F13209A7FB0937C7F3431773
:1017F0002F44C8F80870BDE8F08700BF0010014012
:101800001F85EB512DE9F04105460F4616469846D7
:10181000069C2B681B6837EA03030CBF01230023D7
:10182000B3421ED1B4F1FF3FF3D02CB1FEF7D8FE86
:10183000A0EB08008442ECD22A68D36823F4D0736A
:10184000D3602A68536923F001035361202385F88C
:10185000393085F83A30002385F838300320BDE868
:10186000F0810020BDE8F08158B310B5044690F82F
:1018700039300BB3242384F839302268D36823F439
:101880000053D3602046FFF71BFE2268136923F440
:10189000904313612268536923F02A03536122683D
:1018A000D36843F40053D3600020E063202384F81E
:1018B000393084F83A3010BD80F8383001F026FB1A
:1018C000D8E7012070472DE9F04182B01E4690F81C
:1018D0003930DBB2202B04D00223184602B0BDE819
:1018E000F08104460D469046002955D0002A55D077
:1018F00090F83830012B01D10223EEE7012380F864
:1019000038300023C363212380F83930FEF768FEA6
:101910000746A4F82480A4F8268010E000963B46F1
:10192000002280212046FFF76DFF002838D1226871
:101930002B88C3F3080353602369CBB90235E38CCA
:101940009BB2BBB1E38C9BB2013B9BB2E384A36827
:10195000B3F5805FE2D000963B460022802120460E
:10196000FFF750FFF0B923682A785A600135E6E79F
:101970000135E4E700963B46002240212046FFF770
:1019800041FF034608B10323A7E7202284F839204A
:10199000002284F83820A0E701239EE701239CE77A
:1019A00003239AE7032398E790F83A30DBB2202B21
:1019B00001D002207047D1B1DAB190F83830012B54
:1019C00019D081628285C2850023C363222280F8F8
:1019D0003A2080F8383001684A6942F001024A61D1
:1019E0000168CA6842F49072CA60184670470120C4
:1019F00070470120704702207047704708B50168A2
:101A0000CB6823F04003CB60202380F83930FFF708
:101A1000F4FF002008BD704708B590F83A30DBB2FB
:101A2000222B01D0022008BD8368B3F5805F0FD060
:101A300003690BBB836A5A1C8262026852681A707F
:101A4000C38D9BB2013B9BB2C385F3B1002008BD9F
:101A5000826A036943B903685B68C3F308031380B0
:101A6000836A02338362EBE703685B68DBB213804F
:101A7000836A01338362E3E7826A531C83620368EB
:101A80005B6803F07F031370DAE70268D36823F41E
:101A90009073D3600268536923F0010353612023DC
:101AA00080F83A30FFF7B7FF002008BD704700000C
:101AB00010B5044602681368D168526913F00F002C
:101AC00005D113F0200F02D011F0200F53D10028C0
:101AD00067D012F0010202D111F4907F61D013F0AF
:101AE000010F06D011F4807F03D0E06B40F00100BD
:101AF000E06313F0040F04D01AB1E06B40F0020071
:101B0000E06313F0020F04D01AB1E06B40F0040060
:101B1000E06313F0080F04D01AB1E26B42F0080240
:101B2000E263E26B002A48D013F0200F02D011F0DC
:101B3000200F24D123685B6903F04003E26B12F0AD
:101B4000080F00D13BB32046FFF777FC23685A69A2
:101B500012F0400F1BD05A6922F040025A61636BA9
:101B60008BB11A4A1A65606BFEF7B6FD28B3606B3D
:101B7000036D984710BD2046FFF74EFF10BD20466D
:101B8000FFF74AFFD6E72046FFF790FF10BD20463B
:101B9000FFF78CFF10BD2046FFF788FF0023E363AB
:101BA00010BD13F0800F02D011F0800F06D113F09A
:101BB000400F02D011F0400F04D110BD2046FFF7B6
:101BC0004AFC10BD2046FFF719FFF6E7D11B0008BD
:101BD00008B5806B0023C385C384FFF767FF08BD8A
:101BE00008B500F0A9F9002008BD08B500F09AFB7F
:101BF000012801D000F076FC08BD00F10803436025
:101C00004FF0FF328260C3600361002303607047BE
:101C100000230361704743684B609A688A609A6842
:101C2000516099600861036801330360704730B404
:101C30000D68B5F1FF3F02D000F1080202E0026931
:101C400004E01A4653681C68A542FAD253684B60F8
:101C500099608A605160086103680133036030BC99
:101C60007047036942688168916082684168516089
:101C70005A68904205D00022026118680138186045
:101C8000704782685A60F6E7094B9B6A1B6843B944
:101C9000012343B9064B9A6AD268D2685268DA6265
:101CA00070470023F5E74FF0FF32014BDA627047CF
:101CB000B002002010B50446006B00F091FD2046F4
:101CC00000F08EFD10BD2DE9F04780469946089D35
:101CD000099F0A9C266B02F18042013A06EB8206BC
:101CE00026F0070600230F2B07D8C85CE21882F8FD
:101CF0003400CA5C0AB10133F5E7002384F84330AD
:101D0000062D00D90625E56265644FF0000AC4F887
:101D100048A0201DFFF77CFF04F11800FFF778FFB3
:101D20002461C5F10705A5616462C4F84CA084F87C
:101D300050A04A464146304600F038FB206007B1CB
:101D40003C60BDE8F087000070B5002407E004EBBC
:101D50008402930010481844FFF74FFF0134062C0B
:101D6000F5D90E4C04F1BC063046FFF746FF04F1EE
:101D7000D0052846FFF741FF04F11400FFF73DFFAF
:101D800004F1E400FFF739FF2046FFF736FFA662B3
:101D9000C4F8F85070BD00BFE0020020B00200207F
:101DA00038B5054600F02EFB264BD3F8FC20013257
:101DB000C3F8FC20D3F80031002B38D0214BD3F8E6
:101DC00004314BB91F4BD3F80031DA6AEB6A9A42FF
:101DD00002D81C4BC3F800511A4CD4F80831013317
:101DE000C4F80831EB6A01229A40D4F80C110A4376
:101DF000C4F80C2104F1300003EB83039A00291D81
:101E00001044FFF708FF00F01FFBD4F804316BB15A
:101E1000D4F80031DA6AEB6A9A4207D24FF0805266
:101E2000094B1A60BFF34F8FBFF36F8F38BD054B5F
:101E3000C3F80051D3F8FC30012BCDD1FFF784FF5C
:101E4000CAE700BFB002002004ED00E070B5044610
:101E50000E461F4BD3F81051D3F800010430FFF7A2
:101E600000FF60B91A4BD3F80021D16A012202FAAF
:101E700001F1D3F80C2122EA0102C3F80C21B4F1DC
:101E8000FF3F12D02C44124BD3F800315C60A542C6
:101E900014D80F4DA86AD5F800110431FFF7C7FE1A
:101EA000EB6A9C4200D2EC6270BD002EEAD008487A
:101EB000D0F800110431FFF7AEFE70BD044BD3F82B
:101EC000F800D3F800110431FFF7B1FE70BD00BF78
:101ED000B00200202DE9F04385B006460F461546B6
:101EE0009846900000F0F6FB00B38146542000F0C5
:101EF000F1FB0446B0B1C0F83090CCB1002303939D
:101F000002940D9B01930C9B009343462A4639464D
:101F10003046FFF7D8FE2046FFF742FF012005B00C
:101F2000BDE8F083484600F05BFCE6E70024E4E708
:101F30004FF0FF30F3E7000000B583B0174B01937B
:101F400000230093802216491648FFF7C3FF01289B
:101F500005D0B0F1FF3F17D003B05DF804FB4FF0A0
:101F6000500383F31188BFF36F8FBFF34F8F0E4B76
:101F70004FF0FF32DA620122C3F804210022C3F8D5
:101F8000102100F0DBFAE7E74FF0500383F31188EC
:101F9000BFF36F8FBFF34F8FFEE700BFCC0300206E
:101FA000603200086D220008B0020020034AD2F817
:101FB00018310133C2F81831704700BFB002002059
:101FC0002DE9F041424BD3F81831002B70D1404B32
:101FD000D3F810510135C3F81051CDB99B6A1B6875
:101FE00043B14FF0500383F31188BFF36F8FBFF3FA
:101FF0004F8FFEE7364B9A6AD3F8F8109962C3F810
:10200000F820D3F820210132C3F82021FFF73CFE4D
:102010002F4BDB6A9D423FD200242D4AD2F800317B
:10202000DB6A03EB830399000A44136B012B46D947
:10203000012444E00124264B9B6A1B6873B30023F0
:1020400073BB234B9B6ADB68DE6873689D422CD3AD
:1020500006F104084046FFF704FEB36A1BB106F11F
:102060001800FFF7FEFDF36A01229A40184FD7F8D7
:102070000C110A43C7F80C2107F1300003EB83036E
:102080009A0041461044FFF7C6FDF26AD7F80031C6
:10209000DB6A9A42CED2CEE70024CCE70123CFE719
:1020A0004FF0FF320A4BDA62B7E7094AD362B4E76E
:1020B000074AD2F824310133C2F824310024044BFA
:1020C000D3F8283103B101242046BDE8F08100BFD8
:1020D000B00200203A4BD3F8183143B94FF0500307
:1020E00083F31188BFF36F8FBFF34F8FFEE770B597
:1020F00000F088F9324BD3F81821013AC3F81821BF
:10210000D3F81831002B57D12D4BD3F8FC3023B91D
:10211000002400F099F9204670BD0024284B5B692B
:102120002BB3274D2B6ADC6804F11800FFF799FDEB
:10213000261D3046FFF795FDE36A01229A40D5F847
:102140000C110A43C5F80C2105F1300003EB8303A1
:102150009A0031461044FFF75EFDE26AD5F800317F
:10216000DB6A9A42DAD30122C5F82821D6E70CB1FE
:10217000FFF78AFD124BD3F824417CB9104BD3F8FA
:102180002831DBB14FF080520E4B1A60BFF34F8FF6
:10219000BFF36F8F0124BCE7013C08D0FFF710FFAD
:1021A0000028F9D00122064BC3F82821F4E70022C9
:1021B000034BC3F82421E1E70024AAE70024A8E7A1
:1021C000B002002004ED00E010B5B0B10446104BA1
:1021D000D3F8183143B14FF0500383F31188BFF3A4
:1021E0006F8FBFF34F8FFEE7FFF7E0FE0021204621
:1021F000FFF72CFEFFF76EFF00E0002038B94FF02C
:102200008052044B1A60BFF34F8FBFF36F8F10BD26
:10221000B002002004ED00E038B5134BD3F81431C0
:102220000BB3FFF7C3FE104BD3F8E440FFF752FFA8
:10223000002CF2D000F0E6F80B4CD4F8F030DD685A
:10224000281DFFF70EFDD4F8FC30013BC4F8FC302C
:10225000D4F81431013BC4F8143100F0F5F82846E5
:10226000FFF728FDD9E738BDB002002008B5FFF719
:10227000D3FF064B1B6B012BF9D94FF08052044B57
:102280001A60BFF34F8FBFF36F8FF0E7B0020020EB
:1022900004ED00E0224BD3F81831CBB9204A0023DB
:1022A000C2F82831D2F80C31B3FA83F3DBB2C3F1B0
:1022B0001F0303EB830081000A44126B6AB94FF0DD
:1022C000500383F31188BFF36F8FBFF34F8FFEE787
:1022D0000122134BC3F82821704710B4104A99000B
:1022E000CC18A0001044446B646844633032194435
:1022F000880001460830024494420BD0084903EBA1
:1023000083039A000A44536BDB68C1F800315DF81F
:10231000044B70476068024A0A445063EEE700BF0E
:10232000B0020020064BD3F804312BB1044BD3F894
:1023300018311BB9022070470120704700207047F8
:10234000B00200200B4B1B68B3F1FF3F08D04FF0E9
:10235000500383F31188BFF36F8FBFF34F8FFEE7F6
:102360004FF0500383F31188BFF36F8FBFF34F8F8C
:10237000FEE700BF0800002006480068006880F300
:10238000088862B661B6BFF34F8FBFF36F8F00DF6F
:1023900000BF000008ED00E0DFF80C00016841F428
:1023A000700101607047000088ED00E04FF080731D
:1023B00040F8043C21F0010140F8081C054B40F8AE
:1023C0000C3C40F8202C6FF0020340F8243C4438C9
:1023D000704700BF45230008000000000000000017
:1023E000074B19680868B0E8F04F80F30988BFF31D
:1023F0006F8F4FF0000080F311887047AFF30080BB
:10240000B00300204FF0500383F31188BFF36F8FA8
:10241000BFF34F8F0A4A136801331360012B0DD1AC
:10242000084B1B6813F0FF0F08D04FF0500383F3E5
:102430001188BFF36F8FBFF34F8FFEE7704700BF68
:102440000800002004ED00E0094B1B6843B94FF081
:10245000500383F31188BFF36F8FBFF34F8FFEE7F5
:10246000013B034A13600BB983F31188704700BF27
:102470000800002000000000000000000000000034
:10248000EFF30980BFF36F8F154B1A681EF0100F22
:1024900008BF20ED108A20E9F04F10604DF8043D90
:1024A0004FF0500080F31188BFF34F8FBFF36F8F51
:1024B000FFF7F0FE4FF0000080F3118808BC1968A8
:1024C0000868B0E8F04F1EF0100F08BFB0EC108A9B
:1024D00080F30988BFF36F8F704700BFAFF30080B0
:1024E000B003002008B54FF0500383F31188BFF309
:1024F0006F8FBFF34F8FFFF763FD18B14FF080521E
:10250000024B1A60002383F3118808BD04ED00E03C
:10251000064B1B68064AA2FB03239B09013B054AA5
:1025200013600722044B1A60704700BFC0000020F0
:10253000D34D621014E000E010E000E0314B1A6867
:10254000314B9A4219D02F4B1A68304B9A421DD00A
:1025500000B583B02E4B1A78D2B20192FF221A70C6
:102560001B78DBB28DF803309DF8033003F0500385
:10257000284A1370072353601BE04FF0500383F386
:102580001188BFF36F8FBFF34F8FFEE74FF05003FB
:1025900083F31188BFF36F8FBFF34F8FFEE71D4AA0
:1025A0005368013B53609DF803305B00DBB28DF84C
:1025B00003309DF8033013F0800FF0D1154A5368B3
:1025C0001B0203F4E0635360019BDBB2104A1370FB
:1025D000114B1A6842F470021A601A6842F0704295
:1025E0001A60FFF795FF00220C4B1A60FFF7D4FE2C
:1025F0000B4A136843F040431360FFF7BDFEFFF73B
:10260000A1FE00BF00ED00E071C20F4170C20F419A
:1026100000E400E0DC03002020ED00E008000020E2
:1026200034EF00E0134A12F0070F20D0D11D21F043
:102630000701C1F5705313440A460F49C1F8182920
:102640000020C1F81C091344083B23F00703C1F81C
:10265000203958601860981A50601360C1F8240936
:10266000C1F828094FF00043C1F82C3970474FF4E6
:102670007053E2E7E4030020CC36002010B4134B83
:102680001A6882421CD359685C18A04203D1406882
:1026900001445960184641684418A24214D10C4CB8
:1026A000D4F82049A2420DD05268114441601A6802
:1026B00012680260984200D018605DF8044B7047C1
:1026C0001346DDE70460F5E70260F3E7E43F00202E
:1026D000CC36002070B50446FFF768FC3F4BD3F8BA
:1026E0002039C3B13D4BD3F82C391C426CD1ACB16D
:1026F000083414F0070F11D024F00704083404F054
:1027000007035BB14FF0500383F31188BFF36F8F62
:10271000BFF34F8FFEE7FFF785FFE3E7002C55D0AF
:102720002E4BD3F828399C4252D82C4BD3F8185949
:1027300003F6181301E02B4615466A68944202D945
:102740002A68002AF7D1254AD2F82029954241D09B
:102750001E6808362A681A606B681B1B102B10D97C
:10276000281910F0070F08D04FF0500383F3118899
:10277000BFF36F8FBFF34F8FFEE743606C60FFF7CF
:102780007DFF6968154AD2F828395B1AC2F82839E2
:10279000D2F82429934202D2104AC2F824390F4BAE
:1027A000D3F82C390B436B6000232B60FFF792FCAE
:1027B00016F0070F10D04FF0500383F31188BFF3CA
:1027C0006F8FBFF34F8FFEE70026EFE70026EDE7A0
:1027D0000026EBE70026E9E7304670BDCC36002046
:1027E00098B338B50446A0F1080550F8042C1749F1
:1027F000D1F82C190A4208D14FF0500383F3118805
:10280000BFF36F8FBFF34F8FFEE750F8080C40B156
:102810004FF0500383F31188BFF36F8FBFF34F8FD7
:10282000FEE722EA010244F8042CFFF7BFFB54F84C
:10283000041C064AD2F828390B44C2F82839284625
:10284000FFF71CFFFFF746FC38BD7047CC36002071
:1028500082B000230193064B1A6B42F001021A6307
:102860001B6B03F001030193019B02B0704700BF93
:102870000038024008B5554D00212846FEF75AFDA4
:102880002B68534C22689A626068FFF79DFC2B68A6
:10289000A2689A626068FFF797FC2B68E2689A6208
:1028A0006068FFF791FC2B68A2689A626068FFF786
:1028B0008BFC2B6822689A626068FFF785FC2B68A6
:1028C00022689A626068FFF77FFC2B6822689A6230
:1028D0006068FFF779FC2B68A2689A626068FFF76E
:1028E00073FC2B68A2689A626068FFF76DFC2B6826
:1028F000A2689A626068FFF767FC2B6822689A6298
:102900006068FFF761FC2B6822699A626068FFF7D4
:102910005BFC2B6822699A626068FFF755FC2B68A4
:1029200022689A626068FFF74FFC2B68A2689A627F
:102930006068FFF749FC2B68E2689A626068FFF7FD
:1029400043FC2B68A2689A626068FFF73DFC2B6825
:1029500022689A626068FFF737FC2B6822689A62E7
:102960006068FFF731FC2B6822689A626068FFF7A5
:102970002BFC2B68A2689A626068FFF725FC2B6825
:10298000A2689A626068FFF71FFC2B68A2689A62CF
:102990006068FFF719FC2B6822689A626068FFF78D
:1029A00013FC2B68A2689A626068FFF70DFC2B6825
:1029B000E2689A626068FFF707FC00212846FEF78C
:1029C000DBFC41F28830FFF7FFFB54E7404000207A
:1029D0000C00002010B5224C012221462148FEF7B0
:1029E000E3FF23780D2B0ED01D4C4FF47A73012298
:1029F00021461C48FEF767FF0122214604F1100022
:102A000000F04AFB10BD4FF47A73032216491548B3
:102A1000FEF759FF0022154B1A6006E0104A1A44CF
:102A2000002111710133114A1360104B1B68092BEF
:102A3000F4D90B4800F11001043000F025FB00220E
:102A40000A4B1A6006E0064A1A4400211174013349
:102A5000064A1360054B1B68092BF4D910BD00BF53
:102A6000FC3F00207C400020683200083C400020F1
:102A700010B51C4BDB69ABB11A4C201D00F0DBFA22
:102A8000236A98421CD0174C201D00F0D4FA164B34
:102A9000586000236362E3612362144A1360144A9E
:102AA00013601AE06423112212491348FEF70BFF4A
:102AB0000C4C201D00F0BFFA20620123E36110BD21
:102AC000201D00F0B8FA0028DDD00AE0054A1A44BB
:102AD000002111710133064A1360054B1B68092B55
:102AE000F4D910BDFC3F00200C000020BC400020A9
:102AF0003C400020200000207C40002038B51A4BCC
:102B0000DB69ABB1184C201D00F095FA236A98429E
:102B100028D0164B1D68201D00F08DFA6863002335
:102B20006362E361124A13602362124A136015E084
:102B30004FF47A73142210491048FEF7C4FE0A4C71
:102B4000201D00F078FA20620123E36138BD064AB7
:102B50001A44002111710133064A1360054B1B68AA
:102B6000092BF4D938BD00BFFC3F002040400020B5
:102B7000BC4000203C400020340000207C4000206D
:102B800008B51BE0264C2368DA6842F02002DA60C0
:102B9000DA6842F04002DA60224D6423202205F117
:102BA0003C012046FEF78FFE6423202205F15C01E4
:102BB0002046FEF788FE01221B4B5A621A4B5B6AC5
:102BC000002BDFD0012B0AD0022BF7D1174B1B684B
:102BD000012B22D0022BF1D1FFF790FFEEE7144832
:102BE00000F029FA114B186001380128E6D80222BA
:102BF0000D4B5A6200220F4B1A6006E00A4A1A4433
:102C00000021117101330B4A13600A4B1B68092B19
:102C1000F4D9094A044B5A60D0E7FFF729FFCDE702
:102C20007C4000200C000020FC3F0020BC40002025
:102C3000004000203C40002039393900FEE7000008
:102C400008B50B480B4B03604FF416534360002349
:102C50008360C36003610C2242618361C361FEF73C
:102C600003FE00B908BD4FF4E3710348FFF7E6FF28
:102C70007C400020004400406C32000800B58BB05E
:102C80001B484FF0804303601A4BDB6F4360002307
:102C90008360C822C2600361FEF77CFAC8B90023D2
:102CA0000893099308A91248FEF79EFBB0B9602368
:102CB00001933223029300220392059201A90C484A
:102CC000FEF7BAFA78B90A4800F006F90BB05DF8D9
:102CD00004FB40F2A3110848FFF7B0FF4FF4D57191
:102CE0000548FFF7ABFF40F2B3110348FFF7A6FF1B
:102CF000404000200C0000206C32000800B595B068
:102D0000002200922A4B196C41F0805119641B6C0F
:102D100003F080530093009B019226490B6823F433
:102D2000404343F480430B600B6803F4404301933A
:102D3000019B0223079301210A9110210B910D930E
:102D40000E9208220F925422109211931293139311
:102D500007A8FDF719FF08BB0F2302930221039177
:102D6000002304934FF480520592069302A8FDF7C6
:102D7000A9FDC0B9FDF752FE0F4BA3FB003080093F
:102D8000FDF784FC0420FDF797FC00220F214FF093
:102D9000FF30FDF73DFC15B05DF804FB40F27B1100
:102DA0000648FFF74BFF4FF4C4710448FFF746FF96
:102DB0000038024000700040D34D62106C320008B1
:102DC00000B583B0FDF7E6FBFFF798FFFFF740FD86
:102DD000FFF736FFFFF752FF00240194012500950D
:102DE00023464FF4006208490848FFF773F801943E
:102DF00000952346642206490648FFF76BF8FEF764
:102E0000EFFEFFF799F8FEE77C320008812B0008FF
:102E1000843200087528000810B582B000240094A0
:102E2000214B5A6C42F480425A645A6C02F480423C
:102E30000092009A01941A6C42F080521A641B6C42
:102E400003F080530193019B0320FDF7CFFB224643
:102E500021466FF00B00FDF7DBFB224621466FF0A9
:102E60000A00FDF7D5FB224621466FF00900FDF769
:102E7000CFFB224621466FF00400FDF7C9FB224636
:102E800021466FF00300FDF7C3FB22460F216FF0D0
:102E90000100FDF7BDFB22460F214FF0FF30FDF78B
:102EA000B7FB02B010BD00BF003802400368B3F1A9
:102EB000804F00D0704782B000230193054B1A6CFD
:102EC00042F001021A641B6C03F001030193019BA1
:102ED00002B0EFE7003802400368B3F1804F00D042
:102EE000704700B587B0202301930223029300238B
:102EF000039304930123059301A90348FDF700FC04
:102F000007B05DF804FB00BF000002400268154BEB
:102F10009A4200D0704710B586B00024009403F5A3
:102F2000FA331A6C42F400321A641B6C03F4003357
:102F30000093009B0C23019302230293012303932C
:102F4000032304930723059301A90748FDF7D8FB42
:102F5000224605212620FDF75BFB2620FDF78AFB94
:102F600006B010BD00440040000002407047FEE77C
:102F7000FEE7FEE7FEE7704708B5FDF725FBFEF725
:102F800034FE08BD08B50348FEF792FDFFF722FDA9
:102F900008BD00BF7C4000200F49D1F8883043F4C1
:102FA0007003C1F888300D4B1A6842F001021A60B4
:102FB000002098601A6822F0847222F480321A602D
:102FC000074A5A601A6822F480221A60D8604FF0CB
:102FD00000638B60704700BF00ED00E000380240E6
:102FE00010300024DFF834D0002103E00C4B5B5894
:102FF000435004310B480C4B42189A42F6D30B4A0B
:1030000002E0002342F8043B094B9A42F9D3FFF750
:10301000C3FF00F015F8FFF7D3FE70470000022051
:10302000A833000800000020940200209402002031
:10303000C0400020FEE70A22002100F0C1B80000D5
:1030400070B50D4E0D4CA41BA4100025A54209D14E
:103050000B4E0C4C00F0ECF8A41BA4100025A5426C
:1030600005D170BD56F8253098470135EEE756F882
:10307000253098470135F2E7A0330008A033000857
:10308000A0330008A4330008034611F8012B03F80D
:10309000012B002AF9D1704730B503461C785D1C1E
:1030A00044B912F1FF3204D311F8014B03F8014B7C
:1030B00014B930BD2B46F1E7002AF2D11A70F0E7BF
:1030C0002DE9F84F8046894692461F468B465D465D
:1030D0000A9815F8014B00F089F82044467816F05C
:1030E00008060BD12D2C0BD12C7801260BF10205F3
:1030F00067B1102F14D1302C0AD011E0AB46E6E7AF
:103100002B2C04BF2C780BF10205F1E7302C27D1D2
:103110002B7803F0DF03582B4BD16C781027023546
:10312000002E0CBF6FF000414FF000410022B1FBB8
:10313000F7FE104607FB1E1CA4F13003092B11D823
:103140001C46A7421DDD531C07D0864516D301D16E
:10315000A44513DB00FB0740012215F8014BEBE708
:103160000A27DDE7A4F14103192B01D8373CE8E732
:10317000A4F16103192B04D8573CE2E74FF0FF326A
:10318000EBE7531C08D12223C8F800300846BAF1F7
:10319000000F07D1BDE8F88F06B14042BAF1000F29
:1031A0000CD022B1013DCAF80050BDE8F88F4D4661
:1031B000F9E73024002FB3D10827B1E7BDE8F88F35
:1031C000084B37B51C68084D236A002B08BF2B46F7
:1031D000009313460A4601462046FFF771FF03B0ED
:1031E00030BD00BFC400002028010020D0F8EC0052
:1031F000704782B001B901A942B14BB113780B609D
:103200001278101C18BF012002B070471046FBE76F
:103210006FF00100F8E749B1FF2A85BF8A230360F8
:103220000A704FF0FF3098BF012070470846704782
:10323000F8B500BFF8BC08BC9E467047F8B500BFA3
:08324000F8BC08BC9E46704773
:10324800000000000000000001020304060708094E
:10325800000000000102030449444C45000000003E
:103268000A0D00002E2E2F5372632F6D61696E2E8A
:10327800630000007461736B000000007461736B7D
:10328800310000004300504F534958002E000020E1
:1032980020202020202020202828282828202020FE
:1032A80020202020202020202020202020202088AE
:1032B8001010101010101010101010101010100412
:1032C8000404040404040404041010101010101062
:1032D8004141414141410101010101010101010156
:1032E800010101010101010101011010101010106C
:1032F8004242424242420202020202020202020226
:103308000202020202020202020210101010200041
:1033180000000000000000000000000000000000A5
:103328000000000000000000000000000000000095
:103338000000000000000000000000000000000085
:103348000000000000000000000000000000000075
:103358000000000000000000000000000000000065
:103368000000000000000000000000000000000055
:103378000000000000000000000000000000000045
:103388000000000000000000000000000000000035
:08339800D4CEFF7F010000000C
:0433A000F50100082B
:0433A400D10100084B
:1033A8000100000010000000AAAAAAAA9E000000BE
:1033B800C8000000B1000000C70000008400000041
:1033C80054696D652064656C6179286D7329203AAC
:1033D800000000006272696768746E657373283054
:1033E8002D31303029203A00507265737320312016
:1033F800746F20536574207468652054696D652066
:1034080064656C61790A0D0050726573732032200F
:10341800746F2053657420746865206272696768E8
:10342800746E6573730A0D003400000063000000B9
:1034380069000000760000009500000030000000E0
:1034480074657374696E67202E2E2E005072657332
:1034580073203320746F20746573740A0D000000A4
:103468000024F400C8000020000000000000000054
:103478000000000000000000000000000000000044
:103488000000000000000000000000000000000034
:103498000000000000000000000000000000000024
:1034A8000000000000000000000000000000000014
:1034B8000000000000000000000000000000000004
:1034C80000000000000000004300000000000000B1
:1034D80000000000000000000000000000000000E4
:1034E8000000000000000000430000000000000091
:1034F80000000000000000000000000000000000C4
:103508000000000000000000430000000000000070
:1035180000000000000000000000000000000000A3
:103528000000000000000000430000000000000050
:103538000000000000000000000000000000000083
:103548000000000000000000430000000000000030
:103558000000000000000000000000000000000063
:103568000000000000000000430000000000000010
:103578000000000000000000000000000000000043
:1035880000000000000000004300000000000000F0
:103598000000000000000000000000000000000023
:1035A800000000000000000017320008F331000896
:1035B8000000000096320008943200089532000896
:1035C80095320008953200089532000895320008B7
:1035D80095320008953200089532000895320008A7
:1035E800FFFFFFFFFFFFFFFFFFFFFFFFFFFF0000E1
:1035F8000100415343494900000000000000000059
:1036080000000000000000000000000000000000B2
:103618000000415343494900000000000000000039
:103628000000000000000000000000000000000092
:04363800000000008E
:0400000508002FE5DB
:00000001FF
